:020000023000CC
:10FC000002C0EFC037C1112484B7882369F0982F50
:10FC10009A70923049F081FF02C097EF94BF282E6E
:10FC200080E002D10C94000085E08093810082E0A6
:10FC30008093C00088E18093C1008CE08093C40071
:10FC400086E08093C2008EE0EFD0279A84E023EC18
:10FC50003FEF91E0309385002093840096BBB09BEA
:10FC6000FECF1F9AA8954091C00047FD02C0815069
:10FC700089F7CED0813479F4CBD0C82FDBD0C2380D
:10FC800011F480E004C088E0C13809F083E0B9D005
:10FC900080E1B7D0EECF823419F484E1D3D0F8CF2D
:10FCA000853411F485E0FACF853581F4B1D0E82EA2
:10FCB000AFD0F82E87FF07C08BB781608BBFEE0CEB
:10FCC000FF1CB8D0E5CF8BB78E7FF8CF863579F49F
:10FCD0009FD08D3451F49CD0CBB79AD0C170880F8F
:10FCE0008C2B8BBF81E0AED0CCCF83E0FCCF8436B1
:10FCF00009F046C08DD0C82FD0E0DC2FCC2788D0AB
:10FD0000C82B86D0D82E5E018EEFB81A00E012E024
:10FD10004801EFEF8E1A9E0A7BD0F80180838401A0
:10FD20008A149B04A9F786D0F5E410E000E0DF1602
:10FD300009F150E040E063E0C70153D08701C12CD6
:10FD400092E0D92EF601419151916F0161E0C80115
:10FD500048D00E5F1F4F2297A9F750E040E065E0C2
:10FD6000C7013FD095CF6081C8018E0D9F1D01D185
:10FD70000F5F1F4FF801FE5FC017D107A1F788CFB3
:10FD8000843701F545D0C82FD0E0DC2FCC2740D0F8
:10FD9000C82B3ED0D82E4ED08701F5E4DF120BC021
:10FDA000CE0DDF1DC801DDD02CD00F5F1F4FC01757
:10FDB000D107C1F76DCFF80187918F0122D021972C
:10FDC000D1F766CF853739F435D08EE11AD088E97E
:10FDD00018D081E05CCF813509F073CF88E024D062
:10FDE00070CFFC010A0167BFE895112407B600FC3B
:10FDF000FDCF667029F0452B19F481E187BFE895A6
:10FE000008959091C00095FFFCCF8093C60008959F
:10FE10008091C00087FFFCCF8091C00084FD01C0AD
:10FE2000A8958091C6000895E0E6F0E098E19083FF
:10FE300080830895EDDF803219F088E0F5DFFFCF91
:10FE400084E1DFCFCF93C82FE3DFC150E9F7CF9133
:10FE5000F1CFCF92DF92EF92FF92DC01CB01642FC2
:10FE60006D01EE24FF24CBBEA901FF90EF90DF903F
:10FE7000CF90B7CF2F923F924F925F926F927F9227
:10FE80008F929F92AF92BF92CF92DF92EF92FF92AA
:10FE90000F931F93CF93DF9300D0CDB7DEB7180138
:10FEA000E9826B017C0110E000E029013A014C1865
:10FEB0005D086E087F0846015701840C951CA61C3E
:10FEC000B71C0215130531F489818823A1F188E05C
:10FED000ABDFFFCF30E020E043E0C701B601B9DF80
:10FEE00080E890E09B838A83ABBEF4012791369132
:10FEF000C501B401641975098609970941E0A9DFB4
:10FF00008A819B8101979B838A8392E0890E911C51
:10FF1000A11CB11C8A819B81892B31F730E020E044
:10FF200045E0C701B60195DF9FEFD91AE90AF90A42
:10FF30000F5F1F4FC0CF0F900F900F90DF91CF91A9
:10FF40001F910F91FF90EF90DF90CF90BF90AF90F7
:10FF50009F908F907F906F905F904F903F902F90E9
:10FF60000895F999FECF92BD81BDF89A992780B581
:10FF70000895262FF999FECF1FBA92BD81BD20BDED
:0EFF80000FB6F894FA9AF99A0FBE01960895FA
:02FFFE000008F9
:040000033000FC00CD
:00000001FF
